:100000000EC01DC023C11BC01AC019C018C017C024
:1000100016C015C014C013C028C111C010C01124CF
:100020001FBECFE5D2E0DEBFCDBF20E0A0E6B0E04E
:1000300001C01D92A736B207E1F75DD025C1E0CF20
:1000400067B358B3BB98C39820B52E7F20BD23E07B
:1000500027B946B523E030E0241B31092AF036B534
:1000600023E0231B206801C020E826B9209160000E
:1000700030916100232BB9F448E0369A3699FECFCF
:1000800024B1822F817090E0209160003091610056
:10009000220F331F280F391F309361002093600017
:1000A00025B1415051F716B880B5816080BD67BB5E
:1000B00058BB80916000909161009C01220F331F1A
:1000C000280F391FA90142955295507F5427407F30
:1000D0005427BA01621B730B9B01220F331F220F9F
:1000E000331F820F931F89599E4F90936100809315
:1000F0006000892F089587B38B6087BB88E181BD3D
:1001000011BC80B58E6080BD479AC29AC49A82E2C3
:1001100087B926B583E090E0821B91092AF096B555
:1001200083E0891B806801C080E886B9369A3699D9
:10013000FECF85B18C3C20F4C49881E080936600AA
:1001400016B880B5816080BDAC9A8BB780628BBFDA
:10015000789485B78093650085B7877E806185BF79
:1001600085B7806285BF889585B78F7D85BF10E193
:1001700001E00F2EF7E4EF2EF02D6894FF24F6F83F
:100180008091650085BF809163008823A9F010925B
:10019000630080916400882311F0A89504C011BD0C
:1001A000F1BC0093640085B78093650085B7877EB6
:1001B00085BF109262003AC080916200882309F4E2
:1001C0003DC01092620080916400882319F1109262
:1001D000640086B382958F7080278170C82F80E07D
:1001E000D82F8091660090E0C817D90781F011BD23
:1001F00011BC88B3847F88BB23DF8A3910F0C39A8F
:100200000EC0863610F4C09A0AC0C19A08C011BD4B
:10021000E1BC05C088B3847F88BB11BD11BC85B724
:100220008093650085B7877E806185BF809163007C
:100230008111A6CF809162008111A2CF85B7806223
:1002400085BF889585B78F7D85BF9ACF1F920F9206
:100250000FB60F9211248F9381E0809363008F91EA
:100260000F900FBE0F901F9018951F920F920FB610
:100270000F9211248F9381E0809362008F910F90F1
:0C0280000FBE0F901F901895F894FFCF50
:00000001FF
